:100000000C94380018950000189500001895000011
:10001000189500001895000018950000189500002C
:10002000189500001895000018950000189500001C
:10003000189500001895000018950000189500000C
:1000400018950000189500001895000018950000FC
:1000500018950000189500001895000018950000EC
:1000600018950000189500001895000018950000DC
:100070008FEF8DBFC0EEE8ED4E2E80E18EBFD0E158
:10008000F0E15F2EEEEFFFE0A0E0B1E088278D9376
:100090003197E9F783E08093C40080E08093C50046
:1000A00088E18093C10066248FEF81B9109A109A7D
:1000B00084EF91E00E946C00109884EF91E00E9420
:1000C0006C000C9457003197F1F70895689462F82A
:1000D0000895E89462F80895EF93FF93EE27E82BD4
:1000E000E92B31F0E0EDF7E03197F1F70197D1F727
:0600F000FF91EF9108955D
:00000001FF
